:020000040000FA
:06080000CBEF23F0120013
:06080800BBEF05F0120039
:0608180022EF04F01200C3
:06082A000200E847000097
:10083000DC01000002000000E4470000D6010000D7
:0408400004000000B0
:0C084400D8CFE4FFE0CFE4FFE46EDACF91
:10085000E4FFE2CFDAFFE9CFE4FFEACFE4FFF3CF32
:10086000E4FFF4CFE4FFE6529EA201D19E92030E74
:10087000386E0E50EA6A510FE96E010EEA22EF500F
:10088000385C30E10E50E96EEA6AD890E936EA3613
:10089000690EE926010EEA22EECF38F0EFCF39F0EB
:1008A00039C038F0396A3850D76E0E50E96EEA6AAE
:1008B000D890E936EA36690EE926010EEA22EECF33
:1008C00038F0EFCF39F03850D66EF28AF294D58EE8
:1008D0000E50EA6A510FE96E010EEA22040EEF6E25
:1008E0000E50106E020E386E0F50EA6A510FE96E0C
:1008F000010EEA22EF50385C49E10F50E96EEA6AD6
:10090000D890E936EA36690EE926010EEA22EE5061
:10091000ED1009E10F50EA6A510FE96E010EEA226B
:10092000010EEF6E33D0080E0F5C0CE2070E0F14B1
:10093000386E010E385204E0E846FE0B3806FCE142
:1009400089121AD0100E0F5C0CE2070E0F14386ECD
:10095000010E385204E0E846FE0B3806FCE18A122C
:100960000BD0070E0F14386E010E385204E0E84623
:10097000FE0B3806FCE18B120F50EA6A510FE96E4C
:10098000010EEA22030EEF6E0F500E6E0F2A060EB6
:100990000F5C03E1080E0F6E0AD0130E0F5C03E12B
:1009A000160E0F6E04D0180E0F5C01E10F6A000ED8
:1009B000D8800254000E03542EE2112A000E122297
:1009C0000250115C0350125826E3116A126A030E9A
:1009D000065C1FE20450EA6A480FE96E010EEA2243
:1009E00080CFEFFF0450EA6A4B0FE96E010EEA2256
:1009F00081CFEFFF0450EA6A4E0FE96E010EEA2242
:100A000082CFEFFF042A030E045C01E3046A062A86
:100A100002D0026A036A000ED8800754000E085400
:100A200019E20C50000816E2132A000E1422075097
:100A3000135C085014580EE3136A146A030E0B5C1F
:100A400007E2092A030E095C01E3096A0B2A02D0B6
:100A5000076A086A0C5000080AE2156A1550040D6E
:100A6000F328C26E9E9C9F9C9D8CC280C2829EACCD
:100A70002DD09E9CC4503C6E3CC03DF03C6AC3509F
:100A800000013C103A6E3DC03BF01550060DF3CF0F
:100A900038F0F4CF39F0000E3826010E3922095013
:100AA000020D3850F324E96E3950F420EA6E3AC052
:100AB000EEFF3BC0EDFF152A0C50155C02E39D9C38
:100AC00005D01550040DF328C26EC282F2A442D0A4
:100AD000D59EF294F29A040E386E1050EA6A510FC5
:100AE000E96E010EEA22EF50385C34E1080E105C2A
:100AF0000DE2070E1014386E010E385204E0E8467D
:100B0000FE0B3806FCE1E81C89161CD0100E105CA8
:100B10000DE2070E1014386E010E385204E0E8465C
:100B2000FE0B3806FCE1E81C8A160CD0070E1014E8
:100B3000386E010E385204E0E846FE0B3806FCE140
:100B4000E81C8B161050EA6A510FE96E010EEA227A
:100B5000020EEF6EE552E5CFF4FFE5CFF3FFE5CFF0
:100B6000EAFFE5CFE9FFE5CFDAFFE550E5CFE0FFAB
:100B7000E5CFD8FF1000DACFE4FFE2CFDAFFE6528C
:100B8000E552E5CFDAFF1100D9CFE6FFE1CFD9FF7B
:100B9000020EE126896A92680F0EC16EC2900C6A3D
:100BA000070EB46E8A6A93688B6A94688C6A95683B
:100BB0008D6A9668FC0E8B16FC0E941694840101C7
:100BC000010EBE6F0101DC69DD690A6A096A0B6A00
:100BD000056A046A066A026A036A076A086A116A91
:100BE000126A136A146A156ACA82CA80CA9CCA9AAF
:100BF000CA88CA96FA0ECB6EDF6ADFCF2AF00C0ED7
:100C0000E76E2A18E8AE02D0E73402D0E7502A5C3B
:100C100038E2010EDB6A010EDBCF2AF0030EE76E2D
:100C20002A18E8AE02D0E73402D0E7502A5C27E267
:100C3000DFCF2AF02B6A2ABE2B68060E2B02F3CFD9
:100C40002BF0060E2A02F3CF2AF0F4502B26000ECA
:100C50002A26010E2B22010EDBCF2CF02D6A2CBE92
:100C60002D68D8902C362D362A502C24E96E2B5026
:100C70002D20EA6EEE6AED6A010EDB2ACCD7DF2A60
:100C8000BCD70101B86B0101B96B0101B66B010161
:100C9000B76B0101BA6B0101BB6B0101BC6B0101B8
:100CA000BD6B0E6A0F6A106ADF6ADFCF2AF0180E7A
:100CB000E76E2A18E8AE02D0E73402D0E7502A5C8B
:100CC0001BE2DFCFE9FFEA6AE9BEEA68D890E936BD
:100CD000EA36690EE926010EEA22EE6AED6ADFCFF6
:100CE000E9FFEA6AE9BEEA68510EE926010EEA2246
:100CF000010EEF6EDF2AD9D7D586D59AD59CF2940E
:100D0000F29AF194D08ECA949D829F92F28EF28CC8
:100D1000CA84020EE15C02E2E16AE552E16EE5524C
:100D2000E7CFD9FF1200D9CFE6FFE1CFD9FF020EFE
:100D3000E126010EDB6A0101996BFAEC13F0065013
:100D4000000809E23BEC0BF0052A030E055C01E10B
:100D5000056A0606F4D70B50000809E26DEC0BF0AB
:100D60000A2A030E0A5C01E10A6A0B06F4D70401A1
:100D700004011851800B6CE1060E0101D25D68E39D
:100D80006D50020B65E10101996B040119510101DC
:100D9000995D53E201019951EA6A080FE96E050E67
:100DA000EA22EFCFDFFF0101D6511CE10D0E2A6EC2
:100DB000DF502A5C05E00A0E2B6EDF502B5C12E13F
:100DC0000101010ED66F0101B851EA6A400FE96EC8
:100DD000020EEA220D0EEF6E0101B82BDE52010E5B
:100DE000DD6E15D00D0EDF5C11E00A0EDF5C0EE04B
:100DF0000101B851EA6A400FE96E020EEA22DFCF24
:100E0000EFFF0101D66B0101B82B01D013D0400ECA
:100E10000101B85D02E10101B86B0101B9510101A5
:100E2000B85D02E10D8609D0010EDB5003E01CD94C
:100E3000010EDB6A0101992BA8D70401400E196F3E
:100E4000400E040118170401187D880E04011813C0
:100E50000D5001E181D00DA010D03B0E2A6E420E44
:100E60002B6E2C6A2AC0E6FF2BC0E6FF2CC0E6FFE3
:100E70004DEC22F0E552E552E5520DA210D0350EB0
:100E80002A6E420E2B6E2C6A2AC0E6FF2BC0E6FFAC
:100E90002CC0E6FF4DEC22F0E552E552E5520DA4E0
:100EA00010D0190E2A6E420E2B6E2C6A2AC0E6FF55
:100EB0002BC0E6FF2CC0E6FF4DEC22F0E552E552D8
:100EC000E5520DA610D0FD0E2A6E410E2B6E2C6A37
:100ED0002AC0E6FF2BC0E6FF2CC0E6FF4DEC22F057
:100EE000E552E552E5520DA810D0DE0E2A6E410EF5
:100EF0002B6E2C6A2AC0E6FF2BC0E6FF2CC0E6FF53
:100F00004DEC22F0E552E552E5520DAA00D00DACB1
:100F100010D0BD0E2A6E410E2B6E2C6A2AC0E6FF41
:100F20002BC0E6FF2CC0E6FF4DEC22F0E552E55267
:100F3000E5520DAE10D0A40E2A6E410E2B6E2C6A17
:100F40002AC0E6FF2BC0E6FF2CC0E6FF4DEC22F0E6
:100F5000E552E552E5520D6A35D8020EE15C02E237
:100F6000E16AE552E16EE552E7CFD9FF1200D9CF31
:100F7000E6FFE1CFD9FF0101B651EA6A000FE96E41
:100F8000020EEA22FE0EDBCFEFFF0101B62B400E70
:100F90000101B65D02E10101B66B0101B75101012A
:100FA000B65D01E10D84FE0EDBCF2AF02B6A2ABE6E
:100FB0002B682AC0F3FF2BC0F4FF00D0E552E7CF27
:100FC000D9FF1200D9CFE6FFE1CFD9FFE6520101E8
:100FD0009A5145E1060E0101D25D41E36D50020BCD
:100FE0003EE10101B6510101B75D39E00101B751A0
:100FF0000101D880B6551AE20101B7510101B65D71
:10100000DF6E0101B75101019B6F9C6B000E010166
:101010009B27020E01019C23DFCF9FF10101A06BF2
:101020000101010E9A6FB6C1B7F119D0400E01014E
:10103000D880B755DF6E0101B75101019B6F9C6BE2
:10104000000E01019B27020E01019C23DFCF9FF1BF
:101050000101A06B0101010E9A6F0101B76BE5520E
:10106000E552E7CFD9FF1200D9CFE6FFE1CFD9FF94
:10107000040EE126DE6ADD6A020EDB6A030EDB6A1D
:101080000101B951EA6A400FE96E020EEA22EF50FF
:10109000E66EE66A46EC23F0E552E552020EF3CF27
:1010A000DBFF0101B92B400E0101B95D02E1010135
:1010B000B96B020EDB50DE6EDD6A0101B951EA6ADE
:1010C000400FE96E020EEA22EF502C0835E00101D4
:1010D000B951EA6A400FE96E020EEA22EF500D089C
:1010E0002BE00101B951EA6A400FE96E020EEA22D3
:1010F000EF50E66EE66A46EC23F0E552E552030E49
:10110000F3CFDBFF0101B92B400E0101B95D02E114
:101110000101B96B020EDBCF2CF02CC02DF02C6A34
:10112000030EDB5000012C242A6E000E2D202B6EA6
:101130002AC0DEFF2BC0DDFF000EDBCF1EF0010E4C
:10114000DBCF1FF0490E1E1802E1430E1F1801E10C
:10115000D8D0490E1E1802E1520E1F1801E1CED060
:10116000490E1E1802E1530E1F1801E1C4D0530EA0
:101170001E1802E1430E1F1801E1BAD0530E1E18CB
:1011800002E1520E1F1801E1B0D0530E1E1802E109
:10119000530E1F1801E1A6D0530E1E1802E1420E95
:1011A0001F1801E19CD0430E1E1802E1420E1F18C9
:1011B00001E192D0430E1E1802E1520E1F1801E108
:1011C00088D04F0E1E1802E1420E1F1801E17ED09A
:1011D000570E1E1802E14D0E1F1876E0520E1E1813
:1011E00002E14D0E1F186EE0440E1E1802E1500E73
:1011F0001F1866E04F0E1E1802E1500E1F185DE02A
:10120000490E1E1802E1500E1F1855E0580E1E1808
:1012100002E1540E1F184CE0540E1E1801E11F503D
:1012200045E0410E1E1801E11F503EE0560E1E180B
:1012300001E11F5037E0490E1E1801E11F5030E058
:101240004F0E1E1801E11F5029E0550E1E1802E135
:10125000430E1F1821E0580E1E1802E1430E1F18FE
:1012600018E0430E1E1801E11F5011E0520E1E1827
:1012700001E11F500AE0580E1E1802E1520E1F181D
:1012800001E042D0ABEC0EF07ED0B4D87CD037D9A0
:101290007AD0AEEC0EF077D0B1D875D0A3D973D098
:1012A000EAD971D009DA6FD018DA6DD0E7D86BD0EF
:1012B000A8EC0EF068D0C6DB66D0CCEC0DF063D0A5
:1012C000E3DA61D0A0DA5FD069DA5DD09DEC0FF08F
:1012D0005AD0B1EC0EF057D056EC0FF054D0E4ECED
:1012E00010F051D0A0EC11F04ED0A3EC11F04BD087
:1012F000A6EC11F048D0A9EC11F045D0ACEC11F0FF
:1013000042D0AFEC11F03FD0030EDB501AE1020ED9
:10131000DBCFE6FFE66A020EDBCFE6FFE66A810E70
:101320002A6E410E2B6E2C6A2AC0E6FF2BC0E6FF08
:101330002CC0E6FF4DEC22F02D6E070EE15E2D5025
:1013400021D0030EDBCFE6FFE66A020EDBCFE6FF1D
:10135000E66A030EDBCFE6FFE66A020EDBCFE6FFAE
:10136000E66A590E2A6E410E2B6E2C6A2AC0E6FFE1
:101370002BC0E6FF2CC0E6FF4DEC22F02D6E0B0ECD
:10138000E15E2D5000D00101B951EA6A400FE96ECB
:10139000020EEA22EF500D080DE00D500BE1520E47
:1013A0002A6E2B6ADF502A1803E1DE52DD502B181B
:1013B00001E00D8EB8C1B9F1040EE15C02E2E16A10
:1013C000E552E16EE552E7CFD9FF12000101BE51AF
:1013D00010E0580E2A6E470E2B6E2C6A2AC0E6FFCC
:1013E0002BC0E6FF2CC0E6FF4DEC22F0E552E552A3
:1013F000E5521200C4EC05F0E9DF1200D9CFE6FF98
:10140000E1CFD9FF030EE126010EE66EB2EC11F03A
:10141000E5521D50DF6E020EE66EB2EC11F0E552A1
:10142000DE521DC0DEFF1EC0DDFFDD520D5001E0AB
:101430001BD0DF0418E1D950010FE96EDACFEAFFC3
:10144000EE50ED100BE0010E2A6E2B6A010EDB5000
:101450002A1803E1020EDB502B1804E1010EDBCF4A
:10146000BEF101D00D8CB2DF030EE15C02E2E16A55
:10147000E552E16EE552E7CFD9FF1200D9CFE6FF82
:10148000E1CFD9FF030EE126020EDB6A030EE66E02
:10149000B2EC11F0E5521DC000F01EC001F0010ECB
:1014A000E66EB2EC11F0E552020E1DC0DBFF0D50EE
:1014B00001E01BD0020EDB500CE10050011003E1F3
:1014C000026A036A05D0CA8400C002F001C003F0BA
:1014D0000BD00050011003E1076A086A05D0CA84E6
:1014E00000C007F001C008F071DF030EE15C02E20A
:1014F000E16AE552E16EE552E7CFD9FF1200D9CF9C
:10150000E6FFE1CFD9FF060EE126010EE66EB2EC52
:1015100011F0E5521D50DF6E010EE66EB2EC11F0D7
:10152000E552010E1DC0DBFF010EE66EB2EC11F0BC
:10153000E552020E1DC0DBFF010EE66EB2EC11F0AB
:10154000E552040E1DC0DBFF010EE66EB2EC11F099
:10155000E552050E1DC0DBFF010EE66EB2EC11F088
:10156000E552030E1DC0DBFF0D5001E031D0DF500E
:10157000926E010EDB50936E020EDB50946E040EE1
:10158000DB50956E050EDB50966E030EDB500C089B
:1015900005E20C0EF36E030EF3CFDBFF030EDB5000
:1015A00005E10F0EC16EC2900C6A11D00C6AC26ABE
:1015B000030EDBCFE6FF0F0EE552D880E754C16E75
:1015C000BE0EC06EC280030EDB500C6ECA84FEDEFF
:1015D000060EE15C02E2E16AE552E16EE552E7CF18
:1015E000D9FF1200D9CFE6FFE1CFD9FF050EE126E2
:1015F000010EE66EB2EC11F0E5521D50DF6E010EE9
:10160000E66EB2EC11F0E552010E1DC0DBFF010EDB
:10161000E66EB2EC11F0E552020E1DC0DBFF010ECA
:10162000E66EB2EC11F0E552030E1DC0DBFF010EB9
:10163000E66EB2EC11F0E552040E1DC0DBFF0D505A
:1016400001E00FD0DF50896E010EDB508A6E020E72
:10165000DB508B6E030EDB508C6E040EDB508D6EF8
:10166000B5DE050EE15C02E2E16AE552E16EE552AB
:10167000E7CFD9FF12008450E66EE66A8350E66E2B
:10168000E66A8250E66EE66A8150E66EE66A80504F
:10169000E66EE66A3C0E2A6E410E2B6E2C6A2AC05C
:1016A000E6FF2BC0E6FF2CC0E6FF4DEC22F02D6ECE
:1016B0000D0EE15E2D501200600E2A6E470E2B6E4D
:1016C0002C6A2AC0E6FF2BC0E6FF2CC0E6FF4DECDB
:1016D00022F0E552E552E5521200D9CFE6FFE1CF04
:1016E000D9FFE652DF6A3A0E2A6E410E2B6E2C6A43
:1016F0002AC0E6FF2BC0E6FF2CC0E6FF4DEC22F02F
:10170000E552E552E552DF6A0C50DF5C32E2DFCF92
:101710002AF02B6A2ABE2B68060E2B02F3CF2BF081
:10172000060E2A02F3CF2AF0F4502B26000E2A26AA
:10173000010E2B220A50020D2A50F324E96E2B5081
:10174000F420EA6EEECFE6FFEFCFE6FF340E2C6E0C
:10175000410E2D6E2E6A2CC0E6FF2DC0E6FF2EC076
:10176000E6FF4DEC22F02F6E050EE15E2F50DF2AD2
:10177000CBD75D0E2A6E470E2B6E2C6A2AC0E6FF71
:101780002BC0E6FF2CC0E6FF4DEC22F0E552E552FF
:10179000E552E552E552E7CFD9FF1200D9CFE6FF77
:1017A000E1CFD9FF030EE126030EE66EB2EC11F095
:1017B000E5521DC0DEFF1EC0DDFF010EE66EB2EC7D
:1017C00011F0E552020E1DC0DBFF0D5001E011D0FB
:1017D000DECF2AF0DDCF2BF0000E2A5C100E2B5846
:1017E00007E2DECFE9FFDDCFEAFF020EDBCFEFFF3E
:1017F000EDDD030EE15C02E2E16AE552E16EE552E5
:10180000E7CFD9FF1200D9CFE6FFE1CFD9FF030E12
:10181000E126030EE66EB2EC11F0E5521DC0DEFFCC
:101820001EC0DDFF0D5001E025D0DECF2AF0DDCF58
:101830002BF0000E2A5C100E2B5807E2DECFE9FFDA
:10184000DDCFEAFF020EEFCFDBFF020EDBCFE6FFBC
:10185000E66A2A0E2A6E410E2B6E2C6A2AC0E6FF1B
:101860002BC0E6FF2CC0E6FF4DEC22F02D6E050EDE
:10187000E15E2D50030EE15C02E2E16AE552E16EA9
:10188000E552E7CFD9FF1200D9CFE6FFE1CFD9FF6C
:10189000030EE126050EE66EB2EC11F0E5521D5086
:1018A000DF6E010EE66EB2EC11F0E552010E1DC0C6
:1018B000DBFF010EE66EB2EC11F0E552020E1DC028
:1018C000DBFF0D5001E0B4D0020EDB50010802E254
:1018D0000D8CAED0010EDB50070802E20D8CA8D0B3
:1018E000410E2A6EDF502A5C1CE1020EDB500DE136
:1018F000010EF36E010EDB5004E0D890F336E806DB
:10190000FCE1F350E81C92160BD0010EF36E010EB1
:10191000DB5004E0D890F336E806FCE1F350921275
:1019200086D0420E2A6EDF502A5C1CE1020EDB508C
:101930000DE1010EF36E010EDB5004E0D890F3369A
:10194000E806FCE1F350E81C93160BD0010EF36E91
:10195000010EDB5004E0D890F336E806FCE1F350CA
:10196000931265D0430E2A6EDF502A5C1CE1020EF2
:10197000DB500DE1010EF36E010EDB5004E0D89058
:10198000F336E806FCE1F350E81C94160BD0010E88
:10199000F36E010EDB5004E0D890F336E806FCE16C
:1019A000F350941244D0440E2A6EDF502A5C1CE19E
:1019B000020EDB500DE1010EF36E010EDB5004E070
:1019C000D890F336E806FCE1F350E81C95160BD0EE
:1019D000010EF36E010EDB5004E0D890F336E806FA
:1019E000FCE1F350951223D0450E2A6EDF502A5C9D
:1019F0001CE1020EDB500DE1010EF36E010EDB5017
:101A000004E0D890F336E806FCE1F350E81C9616A3
:101A10000BD0010EF36E010EDB5004E0D890F336CC
:101A2000E806FCE1F350961202D00D8C01D0CEDC1A
:101A3000030EE15C02E2E16AE552E16EE552E7CFB6
:101A4000D9FF1200D9CFE6FFE1CFD9FF030EE1267F
:101A5000020EDB6A050EE66EB2EC11F0E5521D5087
:101A6000DF6E010EE66EB2EC11F0E552010E1DC004
:101A7000DBFF0D5001E086D0010EDB50070802E2CB
:101A80000D8C80D0410E2A6EDF502A5C10E1010ED1
:101A9000F36E010EDB5004E0D890F336E806FCE16B
:101AA000F3508014E76E020EE7CFDBFF56D0420EF4
:101AB0002A6EDF502A5C10E1010EF36E010EDB503E
:101AC00004E0D890F336E806FCE1F3508114E76EA9
:101AD000020EE7CFDBFF41D0430E2A6EDF502A5CB7
:101AE00010E1010EF36E010EDB5004E0D890F336E6
:101AF000E806FCE1F3508214E76E020EE7CFDBFF4D
:101B00002CD0440E2A6EDF502A5C10E1010EF36ED9
:101B1000010EDB5004E0D890F336E806FCE1F35008
:101B20008314E76E020EE7CFDBFF17D0450E2A6E57
:101B3000DF502A5C10E1010EF36E010EDB5004E071
:101B4000D890F336E806FCE1F3508414E76E020EF9
:101B5000E7CFDBFF02D00D8C15D0020EDBCFE6FF06
:101B6000E66A210E2A6E410E2B6E2C6A2AC0E6FF11
:101B70002BC0E6FF2CC0E6FF4DEC22F02D6E050ECB
:101B8000E15E2D50030EE15C02E2E16AE552E16E96
:101B9000E552E7CFD9FF1200D9CFE6FFE1CFD9FF59
:101BA000030EE126050EE66EDDDBE5521D50DF6E0D
:101BB000010EE66ED7DBE552010E1DC0DBFF010E04
:101BC000E66ED0DBE552020E1DC0DBFF0D5001E0DA
:101BD000B5D0020EDB50010802E20D8CAFD0010E31
:101BE000DB50070802E20D8CA9D0410E2A6EDF50AF
:101BF0002A5C1CE1020EDB500DE1010EF36E010EBA
:101C0000DB5004E0D890F336E806FCE1F350E81C22
:101C100089160BD0010EF36E010EDB5004E0D89054
:101C2000F336E806FCE1F350891286D0420E2A6EA4
:101C3000DF502A5C1CE1020EDB500DE1010EF36E59
:101C4000010EDB5004E0D890F336E806FCE1F350D7
:101C5000E81C8A160BD0010EF36E010EDB5004E077
:101C6000D890F336E806FCE1F3508A1265D0430EB3
:101C70002A6EDF502A5C1CE1020EDB500DE1010EE2
:101C8000F36E010EDB5004E0D890F336E806FCE179
:101C9000F350E81C8B160BD0010EF36E010EDB50D7
:101CA00004E0D890F336E806FCE1F3508B1244D000
:101CB000440E2A6EDF502A5C1CE1020EDB500DE15F
:101CC000010EF36E010EDB5004E0D890F336E80607
:101CD000FCE1F350E81C8C160BD0010EF36E010EE4
:101CE000DB5004E0D890F336E806FCE1F3508C12A8
:101CF00023D0450E2A6EDF502A5C1CE1020EDB5019
:101D00000DE1010EF36E010EDB5004E0D890F336C6
:101D1000E806FCE1F350E81C8D160BD0010EF36EC3
:101D2000010EDB5004E0D890F336E806FCE1F350F6
:101D30008D1202D00D8C02D0E6EC09F0030EE15CAE
:101D400002E2E16AE552E16EE552E7CFD9FF120007
:101D5000E6EC09F01200E6EC09F01200E6EC09F0FE
:101D60001200D9CFE6FFE1CFD9FF040EE126050E20
:101D7000E66EF8DAE5521D50DF6E010EE66EF2DA1D
:101D8000E552010E1DC0DBFF030EE66EEBDAE552F5
:101D9000020E1DC0DBFF030E1EC0DBFF0D5001E075
:101DA0007BD0D950020FE96EDACFEAFF720ED880ED
:101DB000EE542E0EED5402E20D8C6ED0D950020F6F
:101DC000E96EDACFEAFFEE50ED101FE02D682E68C5
:101DD0002F6A2D0EE76E020EDBCF30F0030EDBCF45
:101DE00031F0E7503026000E3122326A30502D5C3F
:101DF0002A6E31502E582B6E32502F582C6E020EF8
:101E00002AC0DBFF030E2BC0DBFF010EDB500708EF
:101E100002E20D8C41D0410E2A6EDF502A5C02E1B5
:101E2000DF6A12D0420E2A6EDF502A5C03E1080EF0
:101E3000DF6E0AD0430E2A6EDF502A5C03E1100EDB
:101E4000DF6E02D00D8C28D0010EDB50DF24E96E4E
:101E5000EA6AD890E936EA36690EE926010EEA22E6
:101E6000020EDBCFEEFF030EDBCFEDFF010EDB50EA
:101E7000DF24EA6A510FE96E010EEA22EF040AE15B
:101E8000010EDB50DF24EA6A510FE96E010EEA22EF
:101E9000020EEF6EE6EC09F0040EE15C02E2E16A8C
:101EA000E552E16EE552E7CFD9FF1200D9CFE6FF48
:101EB000E1CFD9FF050EE126010EE66E53DAE552B9
:101EC0001D50DF6E010EE66E4DDAE552020E1DC0AA
:101ED000DBFF010EE66E46DAE552030E1DC0DBFFA6
:101EE000010EE66E3FDAE552010E1DC0DBFF010E6A
:101EF000E66E38DAE552040E1DC0DBFF0D5001E03E
:101F000012D0DFCFB1F1020EDBCFB3F1010EDBCF88
:101F1000B2F1030EDBCFB4F1040EDBCFB5F1B1C1EA
:101F200089FFE6EC09F0050EE15C02E2E16AE552A8
:101F3000E16EE552E7CFD9FF1200D9CFE6FFE1CF3E
:101F4000D9FF040EE126030EDB6A0101B951EA6AEA
:101F5000400FE96E020EEA22EF502C081DE001014D
:101F6000B951EA6A400FE96E020EEA22EF50E66EBE
:101F7000E66AFA0E2A6E400E2B6E2C6A2AC0E6FF25
:101F80002BC0E6FF2CC0E6FF4DEC22F02D6E050EB7
:101F9000E15E2D500D8A0ED10101B92B400E0101D9
:101FA000B95D02E10101B96BB1C189FF0101B21D47
:101FB00089142A6E891C0101B2152A10E76E010EE0
:101FC000E7CFDBFF0101B951EA6A400FE96E020E6B
:101FD000EA22EF500D0801E1EBD00101B951EA6AA4
:101FE000400FE96E020EEA22EF50E66EE66A46EC1A
:101FF00023F0E552E552020EF3CFDBFF300EF36E15
:10200000020EDBCFF4FFF350F45C0FE3020EDB5063
:1020100039080BE3300E2A6E020EDBCFE7FF2A50A1
:10202000E75E020EE7CFDBFF19D0410EF36E020E22
:10203000DBCFF4FFF350F45C0FE3020EDB504608F5
:102040000BE3370E2A6E020EDBCFE7FF2A50E75E66
:10205000020EE7CFDBFF02D00D8CACD0020EDB38D6
:10206000F00BDF6E0101B92B400E0101B95D02E1F9
:102070000101B96B0D0E2A6E0101B951EA6A400FD8
:10208000E96E020EEA22EF502A5C02E10D8892D03E
:102090000101B951EA6A400FE96E020EEA22EF50DF
:1020A000E66EE66A46EC23F0E552E552020EF3CF07
:1020B000DBFF300EF36E020EDBCFF4FFF350F45C67
:1020C0000FE3020EDB5039080BE3300E2A6E020ECE
:1020D000DBCFE7FF2A50E75E020EE7CFDBFF19D028
:1020E000410EF36E020EDBCFF4FFF350F45C0FE30E
:1020F000020EDB5046080BE3370E2A6E020EDBCFD2
:10210000E7FF2A50E75E020EE7CFDBFF02D00D8C1F
:1021100051D0020EDB50DF24DF6E0101B92B400EDF
:102120000101B95D02E10101B96BDF508A6E010E58
:10213000DB50896E0101B55105E0B5C1E6FFD7EC72
:1021400023F0E552B1C189FF0101B45130E0030E23
:10215000B4C1DBFF0101B1510101B3152A6E0101C8
:10216000B35180142A5C0BE1030EDB5008E0000041
:102170000000000000000000030EDB06EBD7030E9A
:10218000B4C1DBFF0101B1510101B3152A6E010198
:10219000B35180142A5C0BE0030EDB5008E0000012
:1021A0000000000000000000030EDB06EBD70AD79A
:1021B000E6EC09F0040EE15C02E2E16AE552E16E50
:1021C000E552E7CFD9FF1200D9CFE6FFE1CFD9FF23
:1021D000050EE126030EDB6A040EDB6A010EE66ED5
:1021E000C1D8E552040E1DC0DBFF040EDB5004E035
:1021F000040EDB50380802E20D8C98D00101B95171
:10220000EA6A400FE96E020EEA22EF502C081DE048
:102210000101B951EA6A400FE96E020EEA22EF505D
:10222000E66EE66AFA0E2A6E400E2B6E2C6A2AC003
:10223000E6FF2BC0E6FF2CC0E6FF4DEC22F02D6E32
:10224000050EE15E2D500D8A71D00101B92B400EB3
:102250000101B95D02E10101B96BB1C189FF010161
:10226000B21D89142A6E891C0101B2152A10E76E6D
:10227000010EE7CFDBFF040EDB5056E00101B95140
:10228000EA6A400FE96E020EEA22EFCFDFFF01019A
:10229000B92B400E0101B95D02E10101B96B040ED9
:1022A000DB06DF508A6E010EDB50896E0101B551ED
:1022B00005E0B5C1E6FFD7EC23F0E552B1C189FFD7
:1022C0000101B45130E0030EB4C1DBFF0101B15193
:1022D0000101B3152A6E0101B35180142A5C0BE190
:1022E000030EDB5008E000000000000000000000CA
:1022F000030EDB06EBD7030EB4C1DBFF0101B151C6
:102300000101B3152A6E0101B35180142A5C0BE060
:10231000030EDB5008E00000000000000000000099
:10232000030EDB06EBD7A7D7E6EC09F0050EE15C60
:1023300002E2E16AE552E16EE552E7CFD9FF120011
:10234000E6EC09F01200E6EC09F01200E6EC09F008
:102350001200E6EC09F01200E6EC09F01200E6ECDF
:1023600009F01200D9CFE6FFE1CFD9FF040EE12634
:10237000030EDB6A0D0E2A6E0101B951EA6A400FA5
:10238000E96E020EEA22EF502A5C05E10D881D6A13
:102390001E6A1F6A93D10101B951EA6A400FE96EC2
:1023A000020EEA22EF502C0820E00101B951EA6A3E
:1023B000400FE96E020EEA22EF50E66EE66AFA0E70
:1023C0002A6E400E2B6E2C6A2AC0E6FF2BC0E6FF59
:1023D0002CC0E6FF4DEC22F02D6E050EE15E2D5077
:1023E0000D8A1D6A1E6A1F6A69D10101B92B400E50
:1023F0000101B95D02E10101B96B2D0E2A6E0101E7
:10240000B951EA6A400FE96E020EEA22EF502A5CE7
:1024100028E1040E2B6EFE0EDB502B5C22E0050E35
:102420002C6EFE0EDB502C5C1CE0FE0EDB0406E086
:10243000030E2A6EFE0EDB502A5C06E10D8C1D6A2F
:102440001E6A1F6A3BD10DD0010EF36E030EF3CF4F
:10245000DBFF0101B92B400E0101B95D02E1010171
:10246000B96B040E2A6EFE0EDB502A5C11E0050EDD
:102470002B6EFE0EDB502B5C0BE0050EE66ED9CF0B
:10248000E6FFDACFE6FF24D9E552E552E5523AD02D
:102490000101B951EA6A400FE96E020EEA22EFCF5C
:1024A0002AF02B6A2C6A2AC0DFFF010E2BC0DBFF4B
:1024B000020E2CC0DBFF050E2A6EFE0EDB502A5CDE
:1024C00019E1000EDBCFE6FF010EDBCFE6FF46ECA5
:1024D00023F0E552E552F3CF2AF0F4CF2BF02C6A2B
:1024E0002BBE2C682AC0DFFF010E2BC0DBFF020EC3
:1024F0002CC0DBFF0101B92B400E0101B95D02E1E7
:102500000101B96B030EDB5021E0DFCF2AF0010E91
:10251000DBCF2BF0020EDBCF2CF02268236824687F
:102520002AC01DF02BC01EF02CC01FF021EC21F0A2
:102530001AC02AF01BC02BF01CC02CF02AC0DFFFF1
:10254000010E2BC0DBFF020E2CC0DBFFFE0EDB50AA
:1025500026E1DFCF2AF0010EDBCF2BF0020EDBCF1E
:102560002CF02C34000E2C1807E6D8807F0E2A544D
:10257000000E2B54000E2C5401E28CD0D9CFE9FF71
:10258000DACFEAFF020ED880EB50FF0A06E6800E93
:10259000EE5CFF0EEE58FF0EEF5801E27BD0FE0E10
:1025A000DB0424E1DFCF2DF0010EDBCF2EF0020E95
:1025B000DBCF2FF02F34000E2F1807E6D880FF0E48
:1025C0002D54000E2E54000E2F5464E3D9CFE9FF92
:1025D000DACFEAFF020ED890EB50000A06E6000EB2
:1025E000EE5C000EEE58000EEF5854E3020E306E13
:1025F000FE0EDB50305C24E1DFCF31F0010EDBCF8B
:1026000032F0020EDBCF33F03334000E331807E61E
:10261000D880FF0E31547F0E3254000E33543AE30B
:10262000D9CFE9FFDACFEAFF020ED880EB50FF0ADC
:1026300006E6000EEE5C800EEE58FF0EEF582AE321
:10264000030E346EFE0EDB50345C29E1DFCF35F033
:10265000010EDBCF36F0020EDBCF37F03734000E41
:10266000371807E6D880FF0E3554FF0E3654000E9B
:10267000375410E3D9CFE9FFDACFEAFF020ED89042
:10268000EB50000A06E6000EEE5C000EEE58000E5F
:10269000EF5805E20D8C1D6A1E6A1F6A0FD0DFCF4E
:1026A0002AF0010EDBCF2BF0020EDBCF2CF02AC07C
:1026B0001DF02BC01EF02CC01FF000D0040EE15CFA
:1026C00002E2E16AE552E16EE552E7CFD9FF12007E
:1026D000D9CFE6FFE1CFD9FF020EE126FD0EDBCF19
:1026E000E9FFFE0EDBCFEAFFEE6AEE6AEE6A010E4C
:1026F000DB6AFC0EDB50F36E010EDBCFF4FFF35010
:10270000F45C55E20101B951EA6A400FE96E020E2C
:10271000EA22EFCFDFFF300EDF5C44E3DF50390801
:1027200041E3FD0EDBCFE9FFFE0EDBCFEAFFEECF8C
:102730002DF0EECF2EF0EFCF2FF00A0E226E236A8F
:10274000246A2DC01DF02EC01EF02FC01FF021ECFA
:1027500021F01AC02DF01BC02EF01CC02FF0300E3F
:10276000DF5C306E316A326A2D5030242A6E2E5072
:1027700031202B6E2F5032202C6EFD0EDBCFE9FF67
:10278000FE0EDBCFEAFF2AC0EEFF2BC0EEFF2CC00F
:10279000EEFF0101B92B400E0101B95D02E101011B
:1027A000B96B02D0000E05D0010EDB2AA2D7010EB4
:1027B00000D02A6E020EE15C02E2E16AE552E16EAF
:1027C0002A50E552E7CFD9FF12000650E66EE66ABE
:1027D000EE0E2A6E400E2B6E2C6A2AC0E6FF2BC02E
:1027E000E6FF2CC0E6FF4DEC22F02D6E050EE15EFB
:1027F0002D5012000101D25108E0010E2A6E6D50D9
:10280000020B01E0010E2A5C22E10101D707000E54
:10281000D85B0101D9510EE10101D751D81109E16D
:102820008B800101D00ED76F070ED86F0101010E0A
:10283000D96F0CD00101D751D81108E18B9001015B
:10284000D00ED76F070ED86F0101D96B5DD0010193
:10285000D2050CE0020E0101D25D08E0030E010179
:10286000D25D04E0050E0101D25D02E18B804CD007
:10287000060E0101D25D48E10101D707000ED85BC9
:102880000101D9510EE10101D751D81109E18B8025
:102890000101100ED76F270ED86F0101010ED96FFD
:1028A00033D00101D9050EE10101D751D81109E159
:1028B0008B900101100ED76F270ED86F0101020E09
:1028C000D96F22D0020E0101D95D0EE10101D7516D
:1028D000D81109E18B800101A00ED76F860ED86F49
:1028E0000101030ED96F10D0030E0101D95D0CE375
:1028F0000101D751D81108E18B900101100ED76F5B
:10290000270ED86F0101D96B120082B403D0010EDB
:0A29100003D002D0000E00D0120028
:06291A00C9EC19F0FB0EF0
:10292000DBCFF3FFDB06F35000090AE017EC1AF0E7
:10293000FA0E82EC1AF0F3E12B1CF1E1010E01D04A
:10294000000EF8EF19F0C9EC19F03B0EE12402E398
:10295000E168E652E16E010EDB6A020EDB6AF90EF7
:10296000DBCFF6FFFA0EDBCFF7FFFB0EDBCFF8FF76
:102970000800F550DF6EDF5002E11CEF19F0250E64
:10298000DF5C02E00FEF19F0030EDB6A040EDB6A76
:10299000050EDB6A060EDB6A070EDB6A31EC19F006
:1029A0002D0EDF5C0CE02B0EDF5C09E0200EDF5CFF
:1029B00006E0230EDF5C03E0300EDF5C1AE1DF503F
:1029C000300A14E0130A0FE0030A0AE00B0A05E0DC
:1029D000060AE4E1030EDB80E1D7030EDB82DED7DB
:1029E000030EDB84DBD7030EDB86D8D7030EDB8830
:1029F000D5D72A0EDF5C1BE12DEC19F07BEC19F02A
:102A000010E0030EDB801E681F68130EDBCF23F07F
:102A1000140EDBCF24F06AEC21F0040E1CC0DBFFA7
:102A200003D0130E64EC19F031EC19F00BD0090E41
:102A3000DB6AD2EC19F003E046EC1AF0FAD7090E83
:102A400064EC19F0030EDBB0DB982E0EDF5C1BE1AB
:102A500031EC19F02A0EDF5C0BE12DEC19F07BEC68
:102A600019F003E1130EB6EC19F031EC19F00BD0AC
:102A7000090EDB6AD2EC19F003E046EC1AF0FAD743
:102A8000090EB6EC19F0680EDF5C07E131EC19F0C5
:102A9000680EDF5C1DE1030E18D0740EDF5C17E0DA
:102AA0007A0EDF5C14E0480EDF5C06E0540EDF5C5B
:102AB00003E05A0EDF5C02E1020E07D06C0EDF5C11
:102AC00003E06A0EDF5C04E1010E09EC1AF0C9DBD9
:102AD000DF506E0A01E17FD31E0A01E192D1200A84
:102AE00001E18FD13F0A01E149D11A0A01E146D142
:102AF0000D0A01E143D1200A01E140D13A0A01E186
:102B00003DD1200A01E13AD1260A01E135D10D0A71
:102B100001E132D11A0A01E1D9D0200A4AE0300A93
:102B20001FE0460A0EE0250A01E083D3D950F90FD1
:102B3000E96EFF0EDA20EA6E010EEE5E000EEE5A2E
:102B4000EE5A17EC1AF0250EE66E95DB03E12B1C0E
:102B500001E169D313EC1AF001E26BD3DB2A69D3EC
:102B6000080EDB6A040EDB50010806E2040EDB04EB
:102B7000DBEC19F0DB508BDB080EDB5009E0030EB9
:102B8000DB50010B05E172DB01E04DD3080EDB6A7F
:102B900064DBEFCFDFFF8BEC1AF003E12B1C01E1CC
:102BA00042D313EC1AF001E3DB2A60DB01E141D3ED
:102BB0003AD3070EDB5002080FE157EC1AF0030E70
:102BC0001EEC1AF00E0EEECFDBFF0F0EEECFDBFF8A
:102BD000100EEECFDBFF20D0F70EDBCF2DF0F80E7E
:102BE000DBCF2EF0020E2D5E000E2E5AF70E2DC0FA
:102BF000DBFFF80E2EC0DBFF2DC0E9FF2EC0EAFF81
:102C00000EEC1AF02C6A0E0E2AC0DBFF0F0E2BC042
:102C1000DBFF100E2CC0DBFF0E0EDBCFE6FF0F0E2E
:102C2000DBCFE6FF100EDBCFE6FF21EC23F0E55211
:102C3000E552E552130E1DC0DBFF140E1EC0DBFF74
:102C4000060EDB5005E0130E52EC1AF001E26ADBCF
:102C500076EC1AF002E2130E37DB39EC1AF006E0DC
:102C6000040E52EC1AF002E2050E2EDB030EDBB06E
:102C700005D0FCDA01E0D7D2080EDB6A090EDB6A68
:102C80000E0EDBCFF6FF0F0EDBCFF7FF100EDBCF04
:102C9000F8FF0800F550DF6EDF5014E07CEC1AF00E
:102CA00011E28BEC1AF003E12B1C01E1BCD2BBDB7F
:102CB00001E3DB2A090EDB2AD9500E0FE96E000E64
:102CC000CBDBE7D7D3DA01E1B4D2ADD2C6DA110E4D
:102CD000EECFDBFF120EEDCFDBFF110EDBCFE6FFF9
:102CE000120EDBCFE6FF13EC23F0E552E552130E94
:102CF000F3CFDBFF140EF4CFDBFF060EDB5004E056
:102D0000130ED0DB01E20EDB76EC1AF002E2130EBA
:102D1000DBDAAFDB05E0040EC5DB02E2050ED4DA38
:102D2000030EDBB005D0A2DA01E07DD2080EDB6A2B
:102D3000090EDB6A110EDBCFE9FF120EDBCFEAFFD3
:102D4000EFCFDFFFDF5014E0D7DB12E2E4DB03E17B
:102D50002B1C01E168D267DB01E3DB2A090EDB2AC9
:102D6000110EDB2ADBCFE9FF120EE8E3DB2AE6D700
:102D70007DDA01E15ED257D2030EDB8E070EDB0453
:102D800010E195DB040E5ADB0A0EEECFDBFF0B0ED3
:102D9000EECFDBFF0C0EEECFDBFF0D0EEECFDBFF39
:102DA0006CD0070EDB5003082CE1030EDBAE0DD018
:102DB000B2DA020E76DAEFCF2AF02B6A2C6A2D6A8D
:102DC0002AAE39D02B682C6835D0F70EDBCF2BF02C
:102DD000F80EDBCF2CF0020E2B5E000E2C5AF70EF5
:102DE0002BC0DBFFF80E2CC0DBFF2BC0E9FF2CC093
:102DF000EAFFEFCF2AF00A0E2AC0DBFF0B0EDB6AD8
:102E000038D0070EDB50020809E1030EDBAE04D018
:102E100059DB2CAE10D00ED055DB0DD0030EDBAE3F
:102E200012D079DA020E3DDAF9DA2C6A2D6A2BAE6D
:102E300002D02C682D68E2DA0C0E2CC0DBFF0D0EE0
:102E40002DC0DBFF1AD0F70EDBCF2CF0F80EDBCF56
:102E50002DF0020E2C5E000E2D5AF70E2CC0DBFF5B
:102E6000F80E2DC0DBFF2CC0E9FF2DC0EAFFD6DA3B
:102E7000C5DA0C0EDB6A0D0EDB6A060EDB5005E1CF
:102E8000010EF36E050EF3CFDBFF150EDB6A160E97
:102E9000DB6AD950370F2A6E000EDA202B6E390EFE
:102EA0002AC0DBFF3A0E2BC0DBFF380EDB6A080EB0
:102EB000DB6A0A0EAEDADF50780A12E0200A10E070
:102EC000280A0CE0200A0AE03F0A06E00D0A02E0A8
:102ED000200A08E1020E05D0080E03D0080EDF26F6
:102EE000100E97DA030EDBBE02D0DB92DB94DB50D0
:102EF000800B24E08ADAD890030EEB50000A08E633
:102F0000000EEE5C000EEE58000EEE58000EEE586D
:102F100015E213DA2168226823682468DBEC22F0CA
:102F20000A0E18C0DBFF0B0E19C0DBFF0C0E1AC017
:102F3000DBFF0D0E1BC0DBFF2D0E08D0030EDBA246
:102F400002D02B0E03D0DBA408D0200EF36E170E98
:102F5000F3CFDBFF150EDB2A02D0170EDB6A050E5E
:102F6000DB5003E1B7D901E189D0C40E2A6E470EC8
:102F70002B6E000E2C6E070EDBCF2DF02E6A2F6A03
:102F8000306A2DC021F02EC022F02FC023F030C0B7
:102F900024F0D3D96CEC23F02A501824F36E2B5074
:102FA0001920F46E2C501A20F86EF4CFF7FFF3CFEF
:102FB000F6FF0800090EF5CFDBFF580EDF5C0FE1CE
:102FC000610EF36E090E7BD90AE3200E2A6E090EFC
:102FD000DBCFE7FF2A50E75E090EE7CFDBFF070EE6
:102FE000DBCF2AF02B6A2C6A2D6A0FDA2AC021F077
:102FF0002BC022F02CC023F02DC024F0EECF1CF00B
:10300000EECF1DF0EECF1EF0EFCF1FF06CEC23F0F3
:103010001FC0EDFF1EC0EDFF1DC0EDFF1CC0EFFF88
:10302000390EDBCFE9FFDB063A0EDBCFEAFF01E228
:10303000DB06090EDBCFEFFF150EDB2A4BD995E13E
:10304000030EDBA61DD06F0EDF5C06E1C1D918E3CD
:10305000150EDB285BDA14D0780EDF5C09E0580E21
:10306000DF5C06E0620EDF5C03E0420EDF5C08E13D
:10307000020EF36E160EF3CFDBFF02D0150EDB6AE5
:10308000030EDB50100B0EE0040EDBCF2AF0050E12
:10309000DB50D8802A5406E2060EDB5003E1040E12
:1030A000DB5034DA95D90AE2050EDBCFE7FF150EC7
:1030B000DB50E75E050EE7CFDBFF02D0050EDB6AD3
:1030C000040EDBCF2AF0160E45D9D8802A5414E21C
:1030D000160EDBCFE6FF150EDBCFE6FF040EDBCFCF
:1030E000E6FF050EDB50E552E75CE552D880E75479
:1030F000E552D880E7545FD9030EDB50010B0BE19A
:10310000080EDB5008E0B2D801E08DD0080EDB508D
:10311000BED8080EDB6A170EDB5007E088D9170E01
:10312000F1D903E12B1C01E17ED0160EDB5016E035
:103130007ED9300EE66E9FD802E12B1C74E077D961
:10314000DFCFE6FF99EC22F0E552E552E552F4CFED
:103150002BF00001F31C02E12B1C65E0050EDBCF18
:103160002AF0160EDB50D8802A5409E2050EDBCF78
:10317000E7FF160EDB50E75E050EE7CFDBFF300EF4
:10318000E66E050ECBD94FE1390EDB2ADBCFE9FF26
:103190003A0E01E3DB2ADBCFEAFF090EEFCFDBFFBC
:1031A000DB500EE044D9090EADD902E12B1C3BE007
:1031B000390EDB2ADBCFE9FF3A0EEDE3DB2AEBD752
:1031C00055D831E1160EDBCFE6FF080EC3D8E55225
:1031D000E7245DD82ED0070EDB50030A1CE0010A5D
:1031E00014E0030A07E07BD9DBCFEEFF020EDBCF52
:1031F000EDFF1FD0F5D82F6A2DAE02D02E682F68B4
:103200002CD8BCD82FC0EEFF14D0EAD82DBE2E6823
:1032100024D8B4D80ED063D9DBCFEFFF0AD07BD946
:1032200005E12B1C03E1F368F46810D0FCD801E33E
:10323000DB2A79D9B8EF14F0010EDBCF2AF0020EA9
:10324000DBCF2BF02AC0F3FF2BC0F4FF3B0EE15C79
:1032500002E2E16AE552E16ECBD029D9020E1EEFFF
:103260001AF061D90800F550DF6E1200200EE66EEC
:10327000080E8EEF1AF099EC22F0E552E552E55275
:10328000F3CF2AF0F4CF2BF00001F31C12002A6ECA
:103290002B6AD950010F4DD92A50EE262B50ED2222
:1032A00012002E5E000E2F5AF70E2EC0DBFFF80E16
:1032B0002FC0DBFF2EC0E9FF2FC0EAFF1200DBCFDB
:1032C000F4FFF350F45C1200DB50E76E040EE7CF1E
:1032D000DBFF12000A0EDBCF2AF00B0EDBCF2BF048
:1032E0000C0EDBCF2CF00D0EDBCF2DF02A502B1067
:1032F0002C102D101200130EEECFDBFF140EEDCFAD
:10330000DBFF130EDBCF2AF0140EDBCF2BF0000116
:10331000800E2B141200F70EDBCF2EF0F80EDBCF51
:103320002FF01200050EDB50E66ED950130F01D9B5
:10333000E552E750EE6EED6A12000A0EDBCF1CF08C
:103340000B0EDBCF1DF00C0EDBCF1EF00D0EDBCF16
:103350001FF01200DBCFE6FF150EDBCFE6FF050EF8
:10336000DB50E552E724E552E7241200DB50CED8CB
:10337000010EF36E060EF3CFDBFF1200EE50EFCF1F
:10338000EAFFE96E2CC0EEFF2DC0EEFF2EC0EEFF6F
:103390001200D9CFE6FFDACFE6FFE1CFD9FFE2CFC7
:1033A000DAFF1200DFCFE6FFE66A5AEC23F0E552BF
:1033B000E552F3501200E76E080EE7CFDBFF120074
:1033C000EECF2AF0EECF2BF0EFCF2CF02D6A1200CB
:1033D000050EDBCF2AF0150EDB50D8802A541200E0
:1033E000010EDBCF2CF0020EDBCF2DF02E6A120087
:1033F000E552E5CFDAFFE7CFD9FF12000A0E2AC067
:10340000DBFF0B0E2BC0DBFF1200D9500A0F99EF28
:103410001AF0F36E070EF3CFDBFF1200EECF2AF0A7
:10342000EFCF2BF01200010EDB2A020E1200FC0E71
:10343000DBCFE6FFFD0EDBCFE6FF12002A5E000EBB
:103440002B5AF70E2AC0DBFFF80E2BC0DBFF2AC079
:10345000E9FF2BC0EAFF1200DA20EA6EEF2AEECF76
:10346000F6FF000EEF22EECFF7FFEF22EECFF8FFD0
:103470001200040EDBCFE6FF130EDB50E552E75CD3
:103480009ADFDB5004DF060EDB501200090EDB5022
:103490000A0DF350DF24D00FE76E090EE7CFDBFFF4
:1034A00031EF19F0DB50F36E050E5FEF19F0F70EF8
:1034B000DBCF2AF0F80EDBCF2BF01200DFCFE6FFD8
:1034C0003BEF19F028DF030EECDEE0EF19F08DEC96
:1034D00014F0E552E552E552E55200091200BDDE56
:1034E000EE50EFCFEAFFE96E010E1200130EDB5033
:1034F000F36E040E5FEF19F0040EDB50F36E090E4D
:103500005FEF19F0DBCFE6FF3BEF19F0E76E050E3A
:10351000E7CFDBFF12008BDF5EEF1AF0DBCFE6FFB9
:1035200086DF67EF1AF0D950F90FE96EFF0E2CEF26
:0C3530001AF0E96E000EDA20EA6E1200BC
:04353C000401205115
:103540001F0B010801E060D004012051600BE8422C
:10355000E842E842E842E842010801E055D00401AF
:10356000245104E00401240501E04ED0040121515E
:10357000230A48E0010A40E0030A30E0010A25E09E
:10358000240A22E0070A1FE0010A1CE0030A11E0F6
:10359000010A01E038D00101030ECB6F0101A90E31
:1035A000CC6F010ECD6F0101D3930101080ED06FD6
:1035B0002BD00101030ECB6F0101A90ECE6F010EBE
:1035C000CF6F22D021D020D01FD00101030ECB6FAE
:1035D0000101A10ECE6F010ECF6F16D00101030EB7
:1035E000CB6F0101A10ECC6F010ECD6F0101D39302
:1035F0000101070ED06F08D00101030ECB6F22C46A
:10360000A8F102D001D000D012000101A16BC20EBE
:10361000A26F010EA36FA46B0101A56B0101A66B44
:103620000101080EA76F01019A6B0101996B1A0E37
:10363000726E1E0E736E0401000E166F050E176F6C
:103640000401400E146F0401400E196F0401080EAE
:103650001A6F050E1B6F0401880E186F0401480EC7
:103660001E6F050E1F6F0401400E1C6F1200D9CF94
:10367000E6FFE1CFD9FF0101996B040118BF39D0F2
:10368000FC0EDBCF2AF004011951D8802A5403E242
:10369000FC0E19C4DBFF0101996BFC0EDB5001012C
:1036A000995D1CE201019951EA6A080FE96E050E65
:1036B000EA22EF50E66E01019951E76EFD0EDBCF75
:1036C000E9FFFE0EDBCFEAFFE750E926000EEA2213
:1036D000E552E750EF6E0101992BDFD70401400E50
:1036E000196F400E040118170401187D880E04019B
:1036F00018130101995100D0E552E7CFD9FF12000C
:10370000D9CFE6FFE1CFD9FFE65201019A5101E09E
:1037100031D0DF6ADF2ADF502A6E2B6A2A5002E19D
:10372000010E2B1801E10BD0FD0EDBCFE9FFDB2AE8
:10373000FE0EDBCFEAFF01E3DB2AEF50EBE1DF50C7
:103740002A6E2B6AD950FD0FE96EFF0EDA20EA6E61
:103750002A50EE5E2B50ED5ADF06FD0EDBCF9BF1BB
:10376000FE0EDBCF9CF1DFCF9FF10101A06B0101C9
:10377000010E9A6FE552E552E7CFD9FF1200D9CF7B
:10378000E6FFE1CFD9FFE65201019A5101E033D0C3
:10379000DF6ADF2ADF502A6E2B6AFF0E2A1801E14A
:1037A0002B5001E10CD0FD0EDBCFF6FFDB2AFE0E25
:1037B000DBCFF7FF01E3DB2A0800F550EAE1DF5039
:1037C0002A6E2B6AD950FD0FE96EFF0EDA20EA6EE1
:1037D0002A50EE5E2B50ED5ADF06FD0EDBCF9BF13B
:1037E000FE0EDBCF9CF1DFCF9FF10101010EA06F38
:1037F0000101010E9A6FE552E552E7CFD9FF1200A1
:10380000D9CFE6FFE1CFD9FFE65204011CBF7DD03E
:10381000030E01019A5D02E101019A6B01019A51C7
:1038200001E173D0020E01019A5D06E104011D6BF6
:103830000101030E9A6F61D001019A055EE1400E0D
:103840002A6E2B6A01019F512A5C000E2B5803E25D
:10385000400EDF6E02D09FC1DFFFDFCF1DF4DF50CF
:1038600001019F5D01019F6F0101480E9D6F050ED3
:103870009E6F0101A00518E1DF5015E09BC1F6FF26
:103880009CC1F7FF0800F5509DC1E9FF9EC1EAFF0A
:10389000EF6E01019D2B000E9E2301019B2B000E5C
:1038A0009C23DF06E9D716D0DF5014E09BC1E9FF67
:1038B0009CC1EAFFEF509DC1E9FF9EC1EAFFEF6E98
:1038C00001019D2B000E9E2301019B2B000E9C23CA
:1038D000DF06EAD701019F5110E104011D512A6E54
:1038E0002B6A400E2A1801E12B5004E10101020E5F
:1038F0009A6F03D00101030E9A6F400E04011C174A
:1039000004011C7D880E04011C13E552E552E7CF2B
:04391000D9FF1200C9
:0C3914006C5002E0000E01D0010E000912
:103920000BE0040100513C0BE842E8420D0802E1C3
:103930000CD801D042D808D06C5002E0000E01D063
:10394000010E040901E04BD81200D9CFE6FFE1CF08
:10395000D9FFE6520101CA6B0101CB6B0101D06BAB
:10396000D16B27EC1EF0DF6ADF502A6E2B6A010E46
:103970002A5C000E2B581BE20101CB5101E017D04D
:10398000F76ADF34FE0BF736F66EF90EF626430EB5
:10399000F7220900F5CF2AF00800F5CF2BF004D06C
:1039A0002BC0FAFF2A50F96EFBDFDF2ADDD7F0D8F3
:1039B000E552E552E7CFD9FF1200020E0101CA5DC0
:1039C0000CE1A4D8040100BD04D00401C80E006FAE
:1039D00003D00401880E006F01D029D91200040E13
:1039E0000101D25D0CE122C46EFF6E50000804E2BA
:1039F0000101050ED26F03D00101030ED26F010148
:103A0000CA050CE10DD8040104BD04D00401C80EA0
:103A1000046F03D00401880E046F01D008D912008E
:103A2000D9CFE6FFE1CFD9FF020EE1260101080E52
:103A3000D05D000ED15905E2D0C1DEFFD1C1DDFF5E
:103A400003D0080EDE6EDD6A0401049304010491C4
:103A5000010EDB5004010413DFCF05F4000EDB5030
:103A60000101D05F010EDB500101D15B0101280E85
:103A7000CE6F040ECF6F0101D3A320D0D9CFE9FFC1
:103A8000DACFEAFFEE50ED1018E0CCC1F6FFCDC161
:103A9000F7FF0800F550CEC1E9FFCFC1EAFFEF6E96
:103AA0000101CE2B000ECF230101CC2B000ECD2324
:103AB000DF06010E01E2DB06E1D71ED0D9CFE9FF18
:103AC000DACFEAFFEE50ED1017E0CCC1E9FFCDC12F
:103AD000EAFFEF50CEC1E9FFCFC1EAFFEF6E01016F
:103AE000CE2B000ECF230101CC2B000ECD23DF0601
:103AF000010E01E2DB06E2D7020EE15C02E2E16ABE
:103B0000E552E16EE552E7CFD9FF1200D9CFE6FFCB
:103B1000E1CFD9FF020EE126030E04010015E76E86
:103B2000010EE7CFDBFF01C4DFFFDE500101D0272C
:103B3000DD500101D1230101280ECC6F040ECD6FA1
:103B4000D9CFE9FFDACFEAFFEE50ED1017E0CCC194
:103B5000E9FFCDC1EAFFEF50CEC1E9FFCFC1EAFFD7
:103B6000EF6E0101CE2B000ECF230101CC2B000EF6
:103B7000CD23DF06010E01E2DB06E2D7020EE15C97
:103B800002E2E16AE552E16EE552E7CFD9FF1200A9
:103B90006D980101CB510FE10401080E016F040182
:103BA000200E026F040E036F0401840E006F0401E7
:103BB000840E046F3BD0040120AF25D00101D05109
:103BC0000401265D0101D1510401275904E226C4F4
:103BD000D0F127C4D1F124DF0101010ECA6F040125
:103BE000080E016F0401200E026F040E036F040122
:103BF000800E006F0401280E066F040E076F04018B
:103C0000C80E046F13D00101020ECA6F0401056BC8
:103C10000401C80E046F0401080E016F0401280E90
:103C2000026F040E036F0401C80E006F1200010141
:103C3000CA6B0401080E016F0401200E026F040E0E
:0E3C4000036F0401880E006F0401046B120074
:023C4E0004016F
:103C50002051600BE842E842E842E842E8420009AD
:103C600001E058D004012151070A53E00B0A51E04A
:103C7000070A42E0010A2CE00B0A28E0020A26E0CB
:103C8000030A22E0080A12E0010A0EE00F0A0AE025
:103C9000030A01E03ED00101010ECB6F0101040EC9
:103CA000D26F38D038D836D093D834D00101010E35
:103CB000CB6F0101D40ECC6F010ECD6F0101D393F8
:103CC0000101010ED06F26D0ABD824D0F9D822D074
:103CD0000101010ECB6F040124510101CC6FCD6BAA
:103CE000D50E0101CC27010E0101CD230101D39393
:103CF0000101010ED06F0ED00101010ECB6F040146
:103D00002451EA6AD50FE96E010EEA2222C4EFFFC0
:103D100001D000D01200800E0401205D58E10401A2
:103D20002351030A34E0010A10E0030A01E04DD0F8
:103D30000101010ECB6F01012E0ECC6F430ECD6F32
:103D4000120E0101D06FD16B40D00101010ECB6F7B
:103D500004012251F66EF76AD890F636F736EF0E68
:103D6000F626430EF7220900F5CFCCF10A00F5CF75
:103D7000CDF1020E0101F76ACC25F66ECD51F72286
:103D80000900F5CFD0F10A00F5CFD1F11ED0010125
:103D9000010ECB6F04012251F66EF76AD890F63609
:103DA000F736F30EF626430EF7220900F5CFCCF1D5
:103DB0000A00F5CFCDF1CCC1F6FFCDC1F7FF080069
:103DC000F5500101D06FD16B00D00101D3831200F7
:103DD0000101010ECB6F0F0EE66E710EE66E0F0E37
:103DE000E66E62EC20F0E552E552E552010EE66E19
:103DF000D50EE66E010EE66E62EC20F0E552E5525D
:103E0000E55222C4D4F10401225104E10101050E5E
:103E1000D26F05D00101060ED26F05EC1BF0120027
:103E20000401286B0401296B040120511F0B020AB5
:103E300014E0030A0EE0010A01E034D00101010E92
:103E4000CB6F040128810101D3A102D00401288392
:103E500029D00101010ECB6F25D00101010ECB6FDE
:103E6000040124510F0B080DF3502B6A000F2A6E2A
:103E7000040E2B2204012451800B01E0010E040DDD
:103E8000F35001012A24CE6F000E2B20CF6FCEC13C
:103E9000E9FFCFC1EAFFEF50040B03E00401010E7C
:103EA000286F00D00101CB050AE10101280ECC6F7B
:103EB000040ECD6F0101D3930101020ED06F1200E9
:103EC0000401220511E1040120511F0B00090CE13E
:103ED0000101010ECB6F030E0401215D03E101011D
:103EE000D38102D00101D391040122513EE10401AA
:103EF00020511F0B020839E1040124510F0B000966
:103F000034E00101010ECB6F040124510F0B080DA9
:103F1000F3502B6A000F2A6E040E2B220401245149
:103F2000800B01E0010E040DF35001012A24CE6F35
:103F3000000E2B20CF6F030E0401215D07E1840EDC
:103F4000CEC1E9FFCFC1EAFFEF6E0FD0040124AF6D
:103F500006D0CEC1E9FFCFC1EAFFEF6A06D0880ED6
:0C3F6000CEC1E9FFCFC1EAFFEF6E1200F6
:043F6C006DA610D856
:103F700002D06DB614D80101D20509E16DBA07D09F
:103F8000686A696A698069880101020ED26F12004D
:103F90006D6A696A6D860101010ED26F12006D6A49
:103FA000696A0101D26B1200FADF12000101D251DD
:103FB00001E13AD06850040B04E06950040B01E0C1
:103FC0003CD86DB231D06850010B04E06950010B50
:103FD00001E056D86850100B04E06950100B01E066
:103FE00024D86850400B04E06950400B01E03DD8F4
:103FF0006850200B04E06950200B01E038D868506D
:10400000020B04E06950020B01E038D8030E0101F5
:10401000D25D01E209D06850080B06E06950080B38
:1040200003E08AEC1CF068961200698468986D823F
:10403000A19AA08A0300A09A12006D9269946894D4
:1040400012000101D3A110D0F8DF6D840101080E28
:10405000DA6F070EDB6F0101DA07000EDB5B01018F
:10406000DA51DB11F8E16D941200689C120070A027
:1040700003D017EC1EF07090689A1200689212003C
:104080006A6A686A9F0E6B6E7B0E696E6E6A0F0EAF
:10409000E66E710EE66E0F0EE66E14D8E552E5522E
:1040A000E552160E706E68A602D06896FCD76D9821
:1040B00017EC1EF00101D3910101D46B0101030E35
:1040C000D26F1200D9CFE6FFE1CFD9FFFD0EDBCFD3
:1040D000E9FFFE0EDBCFEAFFFC0EDB5004E0EE6AE8
:0E40E000FC0EDB06F9D7E552E7CFD9FF120040
:0240EE00537409
:1040F000617475733D25690D0A0021352045727282
:104100003A204E65656420636F6D6D61206E657841
:10411000742C20666F756E643A20272563270D0A7C
:104120000050492C2531750D0A004D522C25303395
:10413000750D0A002C25303475004100492C2530BE
:1041400033692C253033692C253033692C253033E5
:10415000692C253033690D0A002138204572723AE6
:1041600020556E6B6E6F776E20636F6D6D616E6440
:104170002027256325633A253258253258270D0A12
:10418000002138204572723A20556E6B6E6F776E43
:1041900020636F6D6D616E64202725633A25325868
:1041A000270D0A002137204572723A204578747233
:1041B00061207061726D617465720D0A0021362094
:1041C0004572723A20496E76616C69642070617242
:1041D000616D7465722076616C75650D0A0021341D
:1041E000204572723A204D697373696E6720706161
:1041F00072616D657465722873290D0A0021332080
:104200004572723A20525820427566666572206F78
:1042100076657272756E0D0A002132204572723A0F
:1042200020545820427566666572206F76657272FA
:10423000756E0D0A002131200D0A002130200D0A73
:01424000007D
:0E4242001FC029F01EC028F01DC027F01D501F
:104250002202F4CF1BF0F3CF1AF01E502302F4CF4A
:104260001DF0F3CF1CF02202F3501B26F4501C2249
:10427000E86A1D2227502302F3501B26F4501C220B
:10428000E86A1D221F502202F3501C26F4501D2202
:104290001F5023021E6AE86A1E22F3501D26F450A6
:1042A0001E2227502402F3501C26F4501D221F6AA0
:1042B000E86A1E221F2228502402F3501D26F450C3
:1042C0001E22E86A1F2229502402F3501E26F450B1
:1042D0001F22000C1FC029F01EC028F01E50230210
:1042E000F4CF1DF0F3CF1CF01F502402F4CF1FF0C9
:1042F000F3CF1EF02302F3501D26F4501E22E86A6D
:104300001F2228502402F3501D26F4501E22E86A72
:104310001F2224AE90EF21F028501E5E29501F5A14
:0E43200029AE000C23501E5E24501F5A000CC4
:02432E0012017A
:10433000000202000008D8040A0000000102000187
:104340000902430002010080320904000001020258
:1043500001000524001001042402020524060001C6
:104360000524010001070582030800020904010079
:10437000020A00000007050302400000070583024F
:104380004000000403090434034D00690063007217
:10439000006F006300680069007000200054006531
:1043A00000630068006E006F006C006F00670079AA
:1043B00000200049006E0063002E003403430044D7
:1043C0000043002000520053002D00320033003221
:1043D00000200045006D0075006C006100740069EC
:1043E000006F006E002000440065006D006F00400B
:0B43F00043404383438743BB433C35FD
:0443FC002A0EF66E21
:10440000080EF76E000EF86E01010900F550C56F39
:104410000900F550C66F03E1C56701D03DD0090022
:10442000F550C06F0900F550C16F0900F550C26F1B
:1044300009000900F550E96E0900F550EA6E09001F
:1044400009000900F550C36F0900F550C46F090059
:104450000900F6CFC7F1F7CFC8F1F8CFC9F1C0C155
:10446000F6FFC1C1F7FFC2C1F8FF0101C35302E16A
:10447000C45307E00900F550EE6EC307F8E2C40725
:10448000F9D7C7C1F6FFC8C1F7FFC9C1F8FF0101DD
:0A449000C507000EC65BBFD712007F
:06449A00D9CFE6FFDACFE6
:1044A000E6FFE1CFD9FFE2CFDAFFE652E652E6526D
:1044B000E652D950FB0F2A6EFF0EDA202B6E2AC06F
:1044C000DEFFDD6EDECFE6FFDDCFE6FFFB0EDBCFEE
:1044D000E6FFFC0EDBCFE6FFFD0EDBCFE6FFDCC127
:1044E000E6FFDDC1E6FFA3EC14F02A6E070EE15CE7
:1044F00002E2E16AE552E16E2A50020EF3CFDBFFE1
:10450000030EF4CFDBFF020EDBCF2AF0030EDBCF6E
:104510002BF02AC0F3FF2BC0F4FF040EE15C02E293
:10452000E16AE552E16EE552E5CFDAFFE7CFD9FF68
:02453000120077
:0E453200D9CFE6FFDACFE6FFE1CFD9FFE2CF27
:10454000DAFFFB0EDBCF2AF0FC0EDBCF2BF00001F5
:10455000800E2B141AE1FB0EDBCFE9FFFC0EDBCF44
:10456000EAFFEECFF3FFEDCFF4FFEE2A000EEF22CD
:10457000F3CFE9FFF4CFEAFFFD0EDBCFEFFFEF5003
:104580002B6AF36E2BC0F4FF10D0FB0EDB50FE083D
:1045900006E1FD0EDBCFE6FFBDEC23F005D0FD0EFE
:1045A000DBCFE6FFB7EC07F0E552E552E5CFDAFFE7
:0645B000E7CFD9FF120065
:0A45B6001C502102F3CF18F0F4CFDF
:1045C00019F02202F3501926000EF4201A6E1C5026
:1045D0002302F3501A26000EF4201B6E1C502402F6
:1045E000F3501B261D502102F3501926F4501A22B5
:1045F000000E1B221D502202F3501A26F4501B22DB
:104600001D502302F3501B261E502102F3501A2680
:10461000F4501B221E502202F3501B261F50210271
:06462000F3501B261200FE
:0A462600FE0EE3CFE9FFFF0EE3CF25
:10463000EAFFF36AF46AEE5203E0F34AF42AFBD786
:104640001200FF0EE3CFF8FFE552FF0EE3CFF7FFB6
:10465000E552FF0EE3CFF6FFE552E66AE66AE66A48
:104660000900F55209E0FD0EE32A05E1FE0EE32AFA
:1046700002E1FF0EE32AF4D7FD0EE3CF1DF0FE0E9C
:0C468000E3CF1EF0FF0EE3CF1FF012008E
:04468C00FF0EE12418
:10469000E96EFF0EE220EA6EEDCFF4FFEFCFF3FFFD
:1046A000F46607D0600EF36404D07B0EF36001D093
:1046B000F39A1200F36AF46AFF0EE124E96EFF0E2A
:1046C000E220EA6EED6607D02F0EEF6404D03A0EBA
:0846D000EF6001D0F32A120093
:0846D8001B6A1A6A196A186ACC
:1046E000200EE76ED8901C361D361E361F36183643
:1046F00019361A361B362150185C2250195823508F
:104700001A5824501B5809E32150185E2250195A98
:1047100023501A5A24501B5A1C2AE72EE4D71200A1
:1047200005D811D893EC06F0FCD712000F0EC11279
:10473000140E6F6E0101D26B0101D36B0101D46BBA
:10474000C4EC05F01200B6EC1FF06FBE02D0D6EC40
:084750001FF000EC1CF0120048
:084758004F4B0D0A000D0A0091
:1047600055425720465720442056657273696F6E34
:0947700020312E342E330D0A0015
:06477A00FF0EE350ACBA93
:1047800004D0AF6AAB8EAC8A949CACA2FED7AD6E5F
:06479000F36EF46A120052
:0A47960013EE00F023EE00F0F86AC5
:0E47A000179CFEEC21F090EC23F0FDD71200E8
:0247AE00FF0EFC
:1047B000E350E84E1200000000D000D000D0E82EF8
:0447C000FAD7120012
:0C47C40030313233343536373839616219
:0547D000636465660052
:0A47D60000EE00F00F0EEE6AEA623A
:0447E000FDD71200EF
:0447E40000000000D1
:0247E800FEFFD2
:00000001FF
